:0200000480007A
:100000006F000005732F2034930F80006308FF03F7
:10001000930F90006304FF03930FB0006300FF038E
:10002000130F000063040F0067000F00732F2034CC
:1000300063540F006F00400093E19153171F0000BD
:1000400023223FFC171F000023200FFC6FF01FFF2F
:100050009300000013010000930100001302000050
:100060009302000013030000930300001304000038
:100070009304000013050000930500001306000020
:100080009306000013070000930700001308000008
:10009000930800001309000093090000130A0000F0
:1000A000930A0000130B0000930B0000130C0000D8
:1000B000930C0000130D0000930D0000130E0000C0
:1000C000930E0000130F0000930F0000732540F102
:1000D0006310050097020000938202017390523072
:1000E000735044749702000093820201739052305F
:1000F00073500018970200009382020273905230EE
:10010000B70200809382F2FF7390023B9302F001EA
:100110007390023A7350403097020000938242017C
:100120007390523073502030735030309301000080
:1001300097020000938242ED739052301305100035
:100140001315F501634C05000F00F00F930110002B
:100150009308D0051305000073000000930200000F
:10016000638A020073905210B7B20000938292101B
:100170007390223073500030970200009382420146
:1001800073901234732540F17300203093012000E6
:10019000930010001397000093031000631A772652
:1001A0009301300093001000139710009303200078
:1001B000631077269301400093001000139770009E
:1001C00093030008631677249301500093001000F6
:1001D0001397E000B7430000631C7722930160008F
:1001E000930010001397F001B70300806312772289
:1001F000930170009300F0FF139700009303F0FF4A
:1002000063187720930180009300F0FF139710008C
:100210009303E0FF631E771E930190009300F0FFAD
:1002200013977000930300F86314771E9301A000E6
:100230009300F0FF1397E000B7C3FFFF631A771C2A
:100240009301B0009300F0FF1397F001B703008013
:100250006310771C9301C000B720212193801012F6
:1002600013970000B7232121938313126312771A87
:100270009301D000B7202121938010121397100012
:10028000B743424293832324631477189301E00019
:10029000B72021219380101213977000B79390908C
:1002A00093830308631677169301F000B72021218A
:1002B000938010121397E000B7434848631A7714ED
:1002C00093010001B7202121938010121397F001B0
:1002D000B7030080631E7712930110019300100092
:1002E00093907000930300086394701293012001AF
:1002F000130200009300100013977000130307000F
:100300001302120093022000E31652FE930300082A
:10031000631073109301300113020000930010006A
:100320001397E000130000001303070013021200EC
:1003300093022000E31452FEB7430000631A730CCB
:100340009301400113020000930010001397F00185
:100350001300000013000000130307001302120033
:1003600093022000E31252FEB70300806312730A67
:1003700093015001130200009300100013977000C6
:100380001302120093022000E31852FE93030008A8
:1003900063107708930160011302000093001000BE
:1003A000130000001397E0001302120093022000D4
:1003B000E31652FEB7430000631C770493017001FB
:1003C000130200009300100013000000130000004F
:1003D0001397F0011302120093022000E31452FE5F
:1003E000B703008063167702930180019310F00138
:1003F00093030000639E700093019001930010022C
:1004000013904001930300006314700063103002E6
:100410000F00F00F638001009391110093E1110030
:100420009308D00513850100730000000F00F00F42
:10043000930110009308D00513050000730000001D
:10044000731000C000000000000000000000000069
:10045000000000000000000000000000000000009C
:10046000000000000000000000000000000000008C
:0C04700000000000000000000000000080
:1010000000000000000000000000000000000000E0
:1010100000000000000000000000000000000000D0
:1010200000000000000000000000000000000000C0
:1010300000000000000000000000000000000000B0
:081040000000000000000000A8
:040000058000000077
:00000001FF
